:03000000020026D5
:0C002600787FE4F6D8FD75814202006D81
:10012B00013A001121000000000000000000000057
:10013B000000000000000832FEFCFDF9FBF3F7F6AF
:10014B00083BF6F7F3FBF9FDFCFEC101C102C10050
:09015C002CF8E6F5907F057E0009
:10016500D3EF9400EE64809480400B7D6EDDFEEF4E
:060175001F70ED1E80EA80
:01017B002261
:10000E005389F0438901E4F58A758CDCC28DD2A93F
:05001E00D28CD2AF22DC
:03000B00020003ED
:07000300758A00758CDC32E8
:1001D10053877F75985053890F438920758BFD751F
:0B01E1008DFDC2ABD28ED2AFC2AC22AB
:1000F4008B088A09890AAE02AF01EF4E6028C2ACB0
:10010400EDD394004020AF051DEF601AAB08050A3B
:10011400E50AAA097002050914F91201ECF59930EF
:0701240099FDC29980E02261
:10017C008B0B8A0C890DAE02AF01EF4E600E120292
:0D018C0005AD07AB0BAA0CA90D1200F42263
:0300230002021ABC
:05021A00C298C29932F8
:100199007B007A02E4FC743B12015C0CBC08F7EBAF
:0B01A9001B70011AEB4A70ECE4F590AB
:0101B4002228
:1001B5007B007A02E4FC743212015C0CBC08F7EB9C
:0B01C5001B70011AEB4A70ECE4F5908F
:0101D000220C
:1000B2001201D112000E30A00320A11812016120FA
:1000C200001420A006D201D200800B20A108D20089
:1000D200C2028002C20030010BC201C2A2D2A3122C
:1000E200019980D23002CFC202D2A2C2A31201B5BC
:0200F20080C4C8
:100032000200B2E493A3F8E493A34003F68001F232
:1000420008DFF48029E493A3F85407240CC8C333CF
:10005200C4540F4420C8834004F456800146F6DF9E
:10006200E4800B010204081020408090012BE47E02
:10007200019360BCA3FF543F30E509541FFEE49393
:10008200A360010ECF54C025E060A840B8E493A35A
:10009200FAE493A3F8E493A3C8C582C8CAC583CA85
:1000A200F0A3C8C582C8CAC583CADFE9DEE780BE3D
:01015B0000A3
:1001EC00BB010689828A83E0225002E722BBFE0211
:0901FC00E32289828A83E4932244
:10020500E4FFFE1201EC600C0FEF70010E09E970BE
:05021500F20A80EF2257
:00000001FF
